:1000000000308A00E3280000FF00030E8301A600F1
:100010007F08A5000A08AD008A01A50E0408A70004
:100020002008A8002108A9002208AA002308AB0084
:100030002408AC00831383120B1E20288B1833284E
:10004000270884002808A0002908A1002A08A20087
:100050002B08A3002C08A4002D088A00260E83007C
:10006000FF0E7F0E09008A11352881018316861242
:10007000831286160108023C03183A282F08B7009D
:10008000B70803194828000000000000B703402803
:10009000831686128312861201080A3C03184C2824
:1000A00081012E1C94282E108316011383128B10AD
:1000B0000B16C0308B048316061600308312061A06
:1000C0000130003A03195B280108B80083160616B0
:1000D00000308312061A0130013C0319662801081A
:1000E000B90038083902BA003A08023C03187428EB
:1000F0003A08143C031C74281F151F197D281E087C
:10010000A000A00CA00C3F30A0052008A03CA1003E
:1001100038082102AF002F08B0000830A1001F08E6
:10012000C73921049F00CA282E1483160117831291
:100130008B100B16C0308B0483160616003083120A
:10014000061A0130003A03199C280108B8008316EA
:10015000061600308312061A0130013C0319A72845
:100160000108B90038083902BA003A08023C0318FD
:10017000B5283A08143C031CB5282F083002BB00F0
:100180003B08273C031CC4280030A1001F08C739C6
:1001900021049F00CA288B108A1120283530840042
:1001A00000080319E2280130A100A001A00BD62805
:1001B000A10BD5284A30A000A00BDC2800000000CD
:1001C000800BD328003484011F30830583161F144D
:1001D0009F141F159F11FF308312B30083161F1049
:1001E0009F101F119F1183121F179F1783169F13B4
:1001F00083121F149412B3123308831687008312DC
:1002000033163308831687008312B311330883161D
:100210008700003083129400831694000108C039CF
:1002200007388100831290010030A1000538920048
:10023000FF30831692008312331133088316870030
:10024000831207110C309700B31033088316870010
:10025000831287100C309D005A3095009B0064304B
:10026000B500CE200030A1001F08C73921049F002F
:100270000130B500CE208316011783122E141F15EE
:100280001F1940291E08A000A00CA00C3F30A0059B
:100290002008203E1E3EAF002F08B0000B16C030D5
:1002A0008B040430B400FA30B500CE20B40B5329CF
:1002B000331033088316870083120714B3113308F1
:0C02C000831687008312871564296300F1
:02400E00393F38
:00000001FF
